:100000000C9488280C94A5280C94A5280C94A52859
:100010000C94A5280C94A5280C94A5280C94A5282C
:100020000C94A5280C94A7280C94A5280C94A5281A
:100030000C94A5280C94A5280C94E5280C94A528CC
:100040000C94A5280C94A5280C94A5280C94A528FC
:100050000C94A5280C94A5280C94A5280C94A528EC
:100060000C94A5280C94A5280C94A5280C94A528DC
:100070000C94A5280C94A5280C94A5284C656572B1
:10008000746173746520647281636B656E207A7528
:100090006D20466F72747365747A656E2E2E2E0015
:1000A000556E64204C504D2069737420646F6368F2
:1000B000206E81747A6C696368212121004469672C
:1000C0006974616C65204D657373646174656E76E7
:1000D0006572617262656974756E67206D697420FE
:1000E0008162657274616B746574656E204D696BB5
:1000F000726F726563686E65726E00536C696465D9
:100100002020202F2020000D090E5E157116311AB7
:10011000791B731C611D771E3221632278236424AE
:10012000652534263329202A762B662C742D722ED1
:1001300035316E326233683467357A3636392C3A67
:100140006D3B6A3C753D373E38412C426B436944F8
:100150006F45304639492E4A2D4B6C4CF64D704E4A
:10016000DF52E454FC55B45A0A5B2B5D23613C66B4
:100170000869316B346C377030712C72327335749E
:10018000367538792B7A337B2D7C2A7D3900000D2A
:10019000090EB0155116211A591B531C411D571E2B
:1001A000222143225823442445252426A729202AF6
:1001B000562B462C542D522E25314E324233483484
:1001C00047355A3626394C3A4D3B4A3C553D2F3E31
:1001D00028413B424B4349444F453D4629493A4A11
:1001E0005F4B4C4CD64D504E3F52C454DC55605A78
:1001F0000A5B2A5D27613E660869316B346C377093
:1002000030712C7232733574367538792B7A337BB2
:100210002D7C277D3900001EB2154026B33D7B3E64
:100220005B3AB5465D457D4E5C617C5B7E0000209F
:1002300020202020202020202020202020202020BE
:1002400020202020202020202020202020202020AE
:10025000202020202020202020202020202020209E
:10026000202020202020202020202020202020208E
:10027000202020202020202020202020202020207E
:100280002323202020232320202023232323202056
:100290002020232323202020202020202020202055
:1002A000202020202020202020202020202020204E
:1002B000202020202020202020202020202020203E
:1002C000202020202020202020202020202020202E
:1002D0002323202020232320202323202023232006
:1002E0002023232023232020202020202020627967
:1002F00020202020202020202020202020202020FE
:1003000020202020202020202020202020202020ED
:1003100020202020202020202020202020202020DD
:1003200023232020202323202323202020202020BB
:1003300023232020202323202020202020202020B1
:100340004A616E20526F65736C65722020202020F8
:100350002020202020206A616E2E726F65736C65EC
:10036000724074752D62732E646520202020202039
:10037000232320202023232023232020202020206B
:100380002323232323232320202020202020202058
:10039000262053656261737469616E2042728163C5
:1003A0006B6E6572202073652E62727565636B6E6D
:1003B00065724074752D62732E64652020202020A4
:1003C0002323202020232320232320202323232012
:1003D0002323202020232320202020202020202011
:1003E000202020202020202020202020202020200D
:1003F00020202020202020202020202020202020FD
:1004000020202020202020202020202020202020EC
:1004100020232320232320202023232020232320C4
:10042000232320202023232020202020202056307A
:100430002E3030303030303030322020202020201C
:1004400020202020202020202020202020202020AC
:10045000202020202020202020202020202020209C
:100460002020232323202020202023232320232077
:100470002323202020232320202020202020202070
:10048000202020202020202020202020202020206C
:10049000202020202020202020202020202020205C
:1004A000202020202020202020202020202020204C
:1004B000202020202020202020202020202020203C
:1004C000202020202020202020202020202020202C
:1004D000202020202020202020202020202020201C
:1004E000202020202020202020202020202020200C
:1004F00020202020202020202020202020202020FC
:1005000020202020202020202020202020202020EB
:1005100020232323232323202020202020202020C9
:1005200020202020202020202020202020202020CB
:1005300020202023232020202020202020202020B5
:1005400020202020202020202023232320202020A2
:10055000202020202020202020202020202020209B
:100560002023232323232320202020202020202079
:10057000202020202020202020202020202020207B
:10058000202020202020202020202020202020206B
:100590002020202020202020202023232020202055
:1005A000202020202020202020202020202020204B
:1005B0002023202323202320202323232323202020
:1005C000232320232323202023232320232320200D
:1005D0002020232323202020232320232323202003
:1005E00020232323232020202020232320202020F9
:1005F00020202020202020202020202020202020FB
:1006000020202023232020202323202020232320D8
:1006100020232323202323202323232323232320B6
:1006200020202023232020202023232020232320B8
:1006300020202020232320202020232320202020AE
:1006400020202020202020202020202020202020AA
:10065000202020232320202023232323232323207F
:100660002023232020202020232320232023232075
:100670002020202323202020202323202023232068
:100680002023232323232020202023232020202055
:10069000202020202020202020202020202020205A
:1006A000202020232320202023232020202020203E
:1006B0002023232020202020232320232023232025
:1006C0002020202323202020202323202023232018
:1006D0002323202023232020202023232020202008
:1006E000202020202020202020202020202020200A
:1006F00020202323232320202023232323232020DF
:1007000023232323202020202323202320232320CE
:1007100020202323232320202023232020232320C1
:1007200020232323202323202023232323202000CE
:100730002040402D402D2D3A3A20404040402D4051
:100740002D2D3A3A40402D2D2D2D3A3A3A20404059
:1007500020202020202020204040402D2D2020201F
:100760002020404040402D202020202040402D2DA2
:10077000402D20202020404020202020202020200C
:100780004040402D402D2D3A3A3A404040402D40C7
:100790002D2D3A2020402D2D402D3A3A202020208A
:1007A0002020202020202020202020202020202049
:1007B00020204040402D2D2D2D3A203A40404040F1
:1007C0002D2D2D2D3A2040402D2D402D3A3A3A2006
:1007D0002020202020202020202020202020202019
:1007E0002020202040402020202020202020404089
:1007F00020202020202020204040402D402D2D3A38
:100800002020404040402D2D2D2D3A3A40402D2DA6
:100810002D2D3A3A3A204040202020202020202030
:100820004040202020202020202020202020202088
:1008300020202020202020202020202020202020B8
:1008400020202020202020202020202020202020A8
:100850002020202020202020202020202040402D4B
:10086000402D2D3A3A20404040402D2D2D2D3A3A32
:1008700040402D2D402D3A3A2020404020202D4050
:100880002020202040402020402D202020204040BB
:1008900040402D2D2D2D3A3A4040402D402D2D3AEF
:1008A0003A20204040402D2D2D2D3A3A2020202066
:1008B0002020202020202020202020202020202038
:1008C00020402D2D2D2020203A3A404040402D2D13
:1008D00020203A3A4040402D402D20203A204040F0
:1008E0002020404020203A3A404020202D2D202D2D
:1008F0002020404020202D2D2D3A3A3A4040202003
:10090000202D3A2D3A202020202020202D2020208C
:1009100020202020202020202020202020202020D7
:100920002020202020402D2D2D2020203A3A40400C
:1009300040402D2D20203A3A4040402D402D20208F
:100940003A2040402020404020203A3A4040202099
:100950002D2D202D2020404020202D2D2D3A3A3ABB
:1009600040402020202D3A2D3A20202020202020F9
:100970002D2020202020202020202020202020206A
:1009800020202020202020204040402D402D2D3AA6
:10099000203A404040402D2D2D2D3A2040402D2D15
:1009A0002D2D3A3A3A3A404020202D2D2020203A51
:1009B000404020203A2D20203A20404020202D3A4F
:1009C00020203A3A40402020202020203A3A40403F
:1009D0002020202020203A202020202020202020FD
:1009E0002020202020202020202020204040402D9A
:1009F000402D2D3A3A20404040402D402D2D3A3A8E
:100A000040402D2D2D2D3A3A3A20404020202020E4
:100A1000202020204040402D2D202020202040401C
:100A200040402D202020202040402D2D402D2020F2
:100A30002020404020202020202020204040402D09
:100A4000402D2D3A3A3A404040402D402D2D3A203D
:100A500020402D2D402D3A3A2020202020202020FB
:100A60002020202020202020202020202020404046
:100A7000402D402D2D3A203A404040402D2D2D2D27
:100A80003A3A40402D20402D3A3A3A20404020202A
:100A90002D402020203A40402020402D20203A2088
:100AA000404040402D2D2D2D3A3A4040402D402DC4
:100AB0002D3A3A3A20404040202D2D2D3A2020203A
:100AC0002020202020202020202020202020202026
:100AD00020204040402D402D2D20203A40404040D5
:100AE0002D2D2D3A3A2040402D2D2D2D3A2D3A3ADC
:100AF000202020202020203A203A202020202020C2
:100B000020203A2020202020202020203A3A202097
:100B10002020202020203A202020202020202020BB
:100B20003A3A202020202020202020202020202091
:100B30002020202020204040402D402D2D3A203ADA
:100B4000404040402D2D2D2D3A2040402D2D2D2D63
:100B50003A3A3A3A404020202D2D2020203A404079
:100B600020203A2D20203A20404020202D3A2020DD
:100B70003A3A40402020202020203A3A404020208D
:100B8000202020203A20202020202020202020204B
:100B9000202020202020202020204040402D402DBB
:100BA0002D3A3A20404040402D2D2D2D3A3A4040DC
:100BB0002D2D40403A3A2020404020202D2D20204D
:100BC0002020404020202D403A202020404040401E
:100BD000402D2D2D3A3A4040402D2D202D3A3A20DF
:100BE000204040402020202D3A3A20202020202064
:100BF00020202020202020202020202020202020F5
:100C000020202020202020202020202020202020E4
:100C10002020202020202020202020204040402D67
:100C2000402D2D3A3A20404040402D402D2D3A3A5B
:100C300040402D2D2D2D3A3A3A20404020202020B2
:100C4000202020204040402D2D20202020204040EA
:100C500040402D202020202040402D2D402D2020C0
:100C60002020404020202020202020204040402DD7
:100C7000402D2D3A3A3A404040402D402D2D3A200B
:100C800020402D2D402D3A3A2020202020202020C9
:100C90002020202020202020202020202020204034
:100CA000402D402D2D3A3A20404040402D2D2D2DF5
:100CB0003A3A40402D2D402D3A3A20204040202005
:100CC0002D402020202040402020402D202020208A
:100CD000404040402D2D2D2D3A3A4040402D402D92
:100CE0002D3A3A20204040402D2D2D2D3A3A2020FB
:100CF00020202020202020202020202020202020F4
:100D0000202020402D2D2D2D3A3A202040404040DB
:100D1000402D2D2D3A3A4040402D2D2D2D3A3A3A76
:100D200040402020202020203A2040402020202029
:100D30002020203A40402020202020203A3A4040E5
:100D40002020202020203A20404020202020202049
:100D50003A3A20202020202020202020202020205F
:100D60002020202020204040402D402D2D3A3A20A8
:100D7000404040402D2D2D2D3A3A40402D2D402D04
:100D80003A3A2020202020202D4020202020202002
:100D90002020402D20202020404040402D2D2D2D72
:100DA0003A3A4040402D402D2D3A3A2040404040B4
:100DB0002D2D2D2D3A3A20202020202020202020CB
:100DC00020202020202020202020404020202020E3
:100DD0002020202040402020202020202020404093
:100DE000402D402D2D3A2020404040402D2D2D2DCE
:100DF0003A3A40402D2D2D2D3A3A3A2040402020BD
:100E000020202020202040402020202020202020A2
:100E100020202020202020202020202020202020D2
:100E200020202020202020202020202020202020C2
:100E300020202020202020202020202020202020B2
:100E400020204040402D402D2D3A203A4040404047
:100E50002D402D2D3A3A40402D2D402D3A3A3A2042
:100E600040402020202020203A3A404020202020CE
:100E700020203A20404040402D2D2D2D2020404064
:100E8000402D402D2D3A3A3A204040402D2D2D2D19
:100E90003A20202020202020202020202020202038
:100EA0002020202020202040402D402D2D3A3A2087
:100EB000404040402D2D2D2D3A3A40402D2D402DC3
:100EC0003A3A2020404020202D4020202020404041
:100ED0002020402D20202020404040402D2D2D2D31
:100EE0003A3A4040402D402D2D3A3A202040404093
:100EF0002D2D2D2D3A3A202020202020202020208A
:100F00002020202020202020202020402D2D2D209A
:100F100020203A3A404040402D2D20203A3A40408F
:100F2000402D402D20203A204040202040402020CD
:100F30003A3A404020202D2D202D202040402020D6
:100F40002D2D2D3A3A3A40402020202D3A2D3A209E
:100F50002020202020202D20202020202020202084
:100F60002020202020202020202020202020202081
:100F70002020202020202020202020202020202071
:100F80002020202020202020202020204040402DF4
:100F9000402D2D20203A404040402D2D2D3A3A2022
:100FA00040402D2D2D2D3A2D3A3A20202020202072
:100FB000203A203A20202020202020203A202020E3
:100FC0002020202020203A3A2020202020202020ED
:100FD0003A2020202020202020203A3A20202020C3
:100FE0002020202020202020202020202020202001
:100FF0004040402D402D2D3A203A404040402D2D7C
:101000002D2D3A2040402D2D2D2D3A3A3A3A404090
:1010100020202D2D2020203A404020203A2D202035
:101020003A20404020202D3A20203A3A40402020CB
:10103000202020203A3A40402020202020203A2022
:1010400020202020202020202020202020202020A0
:10105000202020204040402D402D2D3A203A404075
:1010600040402D2D2D2D3A3A40402D20402D3A3A2A
:101070003A20404020202D402020203A404020208F
:10108000402D20203A20404040402D2D2D2D3A3A31
:101090004040402D402D2D3A3A3A20404040202DEE
:1010A0002D2D3A202020202020202020202020200C
:1010B00020202020202020204040402D402D2D3A6F
:1010C000203A404040402D2D2D2D3A2040402D2DDE
:1010D0002D2D3A3A3A3A404020202D2D2020203A1A
:1010E000404020203A2D20203A20404020202D3A18
:1010F00020203A3A40402020202020203A3A404008
:101100002020202020203A202020202020202020C5
:101110002020202020202020202020204040402D62
:10112000402D2D3A203A404040402D402D2D3A3A56
:1011300040402D2D402D3A3A3A202040402D20208D
:101140002020202020202D402D2020202020404025
:10115000402D2D2D2D2D202040404040402D2D3A5A
:101160003A3A4040402D2D2D2D2D3A202020202090
:10117000202020202020202020202020202020206F
:10118000202020202020202020202020202020205F
:10119000202020202020202020202020202040400F
:1011A000402D402D2D3A203A404040402D2D2D2DF0
:1011B0003A2040402D2D2D2D3A3A3A3A40402020F9
:1011C0002D2D2020203A404020203A2D20203A206A
:1011D000404020202D3A20203A3A40402020202034
:1011E00020203A3A40402020202020203A20202071
:1011F00020202020202020202020202020202020EF
:1012000020204040402D2D2D2D3A203A4040404096
:101210002D2D2D2D3A2040402D2D402D3A3A3A20AB
:1012200020202020202020202020202020202020BE
:10123000202020204040402D402D2D3A203A404093
:1012400040402D402D2D3A3A40402D2D402D3A3A28
:101250003A202040402D20202020202020202D40FA
:101260002D20202020204040402D2D2D2D2D2020D0
:1012700040404040402D2D3A3A3A4040402D2D2DDF
:101280002D2D3A202020202020202020202020202A
:1012900020202020202020204040402D402D2D3A8D
:1012A0002020404040402D2D2D2D3A3A40402D2DFC
:1012B0002D2D3A3A3A20404020202D2D202020206C
:1012C000404020203A2D20202020404020202D3A50
:1012D000202020204040202020202020202040408E
:1012E00020202020202020202020202020202020FE
:1012F0002020202020202020202020202040402DA1
:10130000402D2D3A3A20404040402D2D2D2D3A3A87
:1013100040402D2D402D3A3A2020404020202D40A5
:101320002020202040402020402D20202020404010
:1013300040402D2D2D2D3A3A4040402D402D2D3A44
:101340003A20204040402D2D2D2D3A3A20202020BB
:10135000202020202020202020202020202020208D
:1013600020402D2D2D2D3A3A202040404040402D48
:101370002D2D3A3A4040402D2D2D2D3A3A3A4040FD
:101380002020202020203A20404020202020202003
:10139000203A40402020202020203A3A404020207F
:1013A000202020203A2040402020202020203A3AAF
:1013B000202020202020202020202020202020202D
:1013C000202020204040402D402D2D3A3A20404002
:1013D00040402D2D2D2D3A3A40402D2D402D3A3AAA
:1013E0002020202020202D402020202020202020D0
:1013F000402D20202020404040402D2D2D2D3A3AD8
:101400004040402D402D2D3A3A20404040402D2D67
:101410002D2D3A3A2020202020202020202020207E
:1014200020202020202020202020202020202020BC
:1014300020202020202020202020202020202020AC
:101440002020202020204040402D402D2D3A3A20C1
:10145000404040402D402D2D3A3A40402D2D2D2D1D
:101460003A3A3A20404020202020202020204040AE
:10147000402D2D2020202020404040402D202020A5
:10148000202040402D2D402D202020204040202095
:101490002020202020204040402D402D2D3A3A3A57
:1014A000404040402D402D2D3A2020402D2D402DF4
:1014B0003A3A2020202020202020202020202020F8
:1014C00020202020202020204040402D402D2D3A5B
:1014D000203A404040402D2D2D2D3A2040402D2DCA
:1014E0002D2D3A3A3A3A404020202D2D2020203A06
:1014F000404020203A2D20203A20404020202D3A04
:1015000020203A3A40402020202020203A3A4040F3
:101510002020202020203A202020202020202020B1
:101520002020202020202020202020204040402D4E
:10153000402D2D3A3A20404040402D2D2D2D3A3A55
:1015400040402D2D402D3A3A2020202020202D40B3
:101550002020202020202020402D2020202040401E
:1015600040402D2D2D2D3A3A4040402D402D2D3A12
:101570003A20404040402D2D2D2D3A3A2020202069
:10158000202020202020202020202020202020205B
:101590004040402D402D2D3A3A20404040402D2DD6
:1015A0002D2D3A3A40402D2D40403A3A20204040DF
:1015B00020202D2D20202020404020202D403A208A
:1015C000202040404040402D2D2D3A3A4040402DB3
:1015D0002D202D3A3A20204040402020202D3A3A1C
:1015E00020202020202020202020202020202020FB
:1015F00020202020202020202020202020202020EB
:1016000020202020202020202020202020202020DA
:10161000202020402D2D2D2020203A3A40404040CF
:101620002D2D20203A3A4040402D402D20203A20B8
:1016300040402020404020203A3A404020202D2D9C
:10164000202D2020404020202D2D2D3A3A3A404098
:101650002020202D3A2D3A202020202020202D202F
:10166000202020202020202020202020202020207A
:101670002020202020204040402D402D2D3A2020A9
:10168000404040402D2D2D2D3A3A40402D2D4040D8
:101690003A3A3A2040402020402D2020202040404F
:1016A00020202D2D2020202040404040402D202073
:1016B00020204040402D2D20202020202040404050
:1016C000202020202020202020202020202020201A
:1016D000202020202020202020202040402D402D90
:1016E0002D3A3A20404040402D2D2D2D3A3A404091
:1016F0002D2D402D3A3A2020404020202D40202002
:10170000202040402020402D2020202040404040EC
:101710002D2D2D2D3A3A4040402D402D2D3A3A2086
:10172000204040402D2D2D2D3A3A202020202020F1
:101730002020202020202020202020202020204089
:101740002D2D2D2020203A3A404040402D2D2020A4
:101750003A3A4040402D402D20203A204040202061
:10176000404020203A3A404020202D2D202D20209E
:10177000404020202D2D2D3A3A3A40402020202D67
:101780003A2D3A202020202020202D20202020200B
:101790002020202020202020202020202020202049
:1017A000202020402D2D2D2020203A3A404040403E
:1017B0002D2D20203A3A4040402D402D20203A2027
:1017C00040402020404020203A3A404020202D2D0B
:1017D000202D2020404020202D2D2D3A3A3A404007
:1017E0002020202D3A2D3A202020202020202D209E
:1017F00020202020202020202020202020202020E9
:101800002020202020204040402D402D203A203A0A
:10181000404040402D2D202D3A3A40402D20402D73
:10182000203A3A2020202020202020202020202084
:1018300020202020202020202020202020202020A8
:101840002020202020202020202020202020202098
:101850002020202020202020202020202020202088
:101860002020202020202020202020202020202078
:101870002020202020202020202020202020202068
:101880002020202020202020202020202020202058
:101890002020202020202020202020202020202048
:1018A0002020202020202020202020202020202038
:1018B0002020202020202020202020202020202028
:1018C0002020202020232320202023232020202309
:1018D00023232320202020232323202020202020F6
:1018E00020202020202020202020202020202020F8
:1018F00020202020202020202020202020202020E8
:1019000020202020202020202020202020202020D7
:1019100020202020202323202020232320202323B5
:1019200020202323202023232023232020202020A5
:10193000202020627920202020202020202020200C
:101940002020202020202020202020202020202097
:101950002020202020202020202020202020202087
:101960002020202020232320202023232023232065
:10197000202020202023232020202323202020205B
:1019800020202020204A616E20526F65736C6572A2
:1019900020202020202020202020206A616E2E720E
:1019A0006F65736C65724074752D62732E6465206B
:1019B0002020202020232320202023232023232015
:1019C0002020202020232323232323232020202002
:1019D0002020202020262053656261737469616E87
:1019E00020427281636B6E6572202073652E627275
:1019F0007565636B6E65724074752D62732E6465D8
:101A000020202020202323202020232320232320C4
:101A100020232323202323202020232320202020B1
:101A200020202020202020202020202020202020B6
:101A300020202020202020202020202020202020A6
:101A40002020202020202020202020202020202096
:101A50002020202020202323202323202020232374
:101A60002020232320232320202023232020202064
:101A700020202056302E3030303030303030322080
:101A80002020202020202020202020202020202056
:101A90002020202020202020202020202020202046
:101AA000202020202020202323232020202020232A
:101AB0002323202320232320202023232020202011
:101AC0002020202020202020202020202020202016
:101AD0002020202020202020202020202020202006
:101AE00020202020202020202020202020202020F6
:101AF00020202020202020202020202020202020E6
:101B000020202020202020202020202020202020D5
:101B100020202020202020202020202020202020C5
:101B200020202020202020202020202020202020B5
:101B300020202020202020202020202020202020A5
:101B40002020202020202020202020202020202095
:101B50002020202020202323232323232020202073
:101B60002020202020202020202020202020202075
:101B7000202020202020202023232020202020205F
:101B8000202020202020202020202020202023234F
:101B90002320202020202020202020202020202042
:101BA0002020202020202323232323232020202023
:101BB0002020202020202020202020202020202025
:101BC0002020202020202020202020202020202015
:101BD0002020202020202020202020202020202302
:101BE00023202020202020202020202020202020F2
:101BF00020202020202023202323202320202323D3
:101C000023232320202323202323232020232323B3
:101C100020232320202020232323202020232320AF
:101C2000232323202020232323232020202020239C
:101C300023202020202020202020202020202020A1
:101C40002020202020202020232320202023232088
:101C50002020232320202323232023232023232366
:101C6000232323232020202023232020202023235C
:101C70002020232320202020202323202020202355
:101C80002320202020202020202020202020202051
:101C90002020202020202020232320202023232335
:101CA000232323232020232320202020202323201C
:101CB000232023232020202023232020202023230F
:101CC00020202323202023232323232020202023FC
:101CD0002320202020202020202020202020202001
:101CE00020202020202020202323202020232320E8
:101CF00020202020202023232020202020232320D8
:101D000023202323202020202323202020202323BE
:101D100020202323202323202023232020202023AE
:101D200023202020202020202020202020202020B0
:101D30002020202020202023232323202020232391
:101D40002323232020232323232020202023232078
:101D50002320232320202023232323202020232368
:101D60002020232320202323232023232020232358
:101D7000232320202020202020202020202020205D
:101D80002020202020202020202020202020202053
:101D90002020202020202020202020202020202043
:101DA0002020202020202020202020202020202033
:101DB0002020202020202020202020202020202023
:101DC0002020202020202020202020202020202013
:101DD0002020202020202020202020202020202BF8
:101DE0002D2D2D2D2D2B20202020202020202020A7
:101DF00020202020202020202020202020202020E3
:101E000020202020202020202020202020202020D2
:101E100020202020202020202020202020202020C2
:101E20002020202020202020202020202020207C56
:101E300020204D20207C2020202020202020202019
:101E40002020202020202020202020202020202092
:101E50002020202020202020202020202020202082
:101E60002020202020202020202020202020202072
:101E70002020202020202020202020202020207C06
:101E800020204120207C20202020202020202020D5
:101E90002020202020202020202020202020202042
:101EA0002B2D2D2D2D2D2D2D2D2D2D2D2D2D2D2B66
:101EB0002020202020202020202020202052532DB0
:101EC000323332203C2D2D2D2032202D2D3E2D2B36
:101ED00020205820202B2D2D2D2D2D2B2020202073
:101EE00020202020202020202020202020202020F2
:101EF0007C202032302F3235204D687A2020207C03
:101F000020202020202020202020202020202020D1
:101F10002020202020202020202020202020207C65
:101F200020203220207C20202020207C20202020E7
:101F300020202020202020202020202020202020A1
:101F40007C20204F737A696C6C61746F7220207CE6
:101F50002020202020202020202020202020202081
:101F60002020202020202020202020202020207C15
:101F700020203320207C20202020207C2020202096
:101F80002020202020202020202020202020202051
:101F90002B2D2D2D2D2D2D2D2B2D2D2D2D2D2D2B77
:101FA0002020202020202020202020202020202031
:101FB0002020202020202020202020202020207CC5
:101FC00020203220207C2020202020322020202091
:101FD0002020202020202020202020202020202001
:101FE00020202020202020207C2020202020202095
:101FF00020202020202020202020202020202020E1
:102000002020202020202020202020202020202BC5
:102010002D2D2D2D2D2B20202020207C2020202018
:1020200020202020202020202020202020202020B0
:10203000202020202020202031202020202020208F
:102040002020202020202020202020202020202090
:102050002020202020202020202020202020202080
:1020600020202020202020202020207C2020202014
:102070002020202020202020202020202020202060
:1020800020202020202020207C20202020202020F4
:102090002020202020202020202020202020202040
:1020A0002020202020202020202020202020202030
:1020B00020202020202020202020207C20202020C4
:1020C0002020202020202020202020202020202010
:1020D00020202020202020207C20202020202020A4
:1020E00020202020202020202020202020202020F0
:1020F0002020202020202020202020202020202BD5
:102100002B3D3D3D3D3D3D3D3D3D3D2B3D3D3D3D23
:102110003D3D3D3D3D3D3D3D3D3D3D3D3D3D3D3DEF
:102120003D3D3D2B2B2020207C20202020202020E6
:10213000202020202020202020202020202020209F
:102140002020202020202020202020202020207C33
:102150007C20202020202020202020202020202023
:10216000202020202020202020202020202020206F
:102170002020207C7C2020207C202020202020204B
:10218000202020202020202020202020202020204F
:102190002020202020202020202020202020207CE3
:1021A0007C202020202020202020202020202020D3
:1021B000202020202020202020202020202020201F
:1021C0002020207C7C2020207C20202020202020FB
:1021D0002020202020202020202020202050532F8D
:1021E00032202D2D2D2D2D2D2032202D2D3E2D2B2D
:1021F0002B20202020202020202020202041546D32
:102200006567613634345020202020202020202093
:102210002020207C3C2D2D2D2B2020202020202014
:1022200020202020202020202020202020202020AE
:102230002020202020202020202020202020207C42
:102240007C20202020202020202020202020202032
:10225000202020202020202020202020202020207E
:102260002020207C7C2020207C202020202020205A
:10227000202020202020202020202020202020205E
:102280002020202020202020202020202020207CF2
:102290007C202020202020202020202020202020E2
:1022A000202020202020202020202020202020202E
:1022B0002020207C7C2020207C202020202020200A
:1022C000202020202020202020202020202020200E
:1022D0002020202020202020202020202020202BF3
:1022E0002B3D3D3D3D3D3D3D3D3D2B3D3D3D3D3D42
:1022F0003D3D3D3D3D2B2B2B2B3D3D3D3D3D3D3D56
:102300003D3D3D2B2B2020207C2020202020202004
:1023100020202020202020202020202020202020BD
:1023200020202020202020202020202020202020AD
:10233000202020202020202020207C202020202041
:1023400020202020207C7C7C7C202020202020201D
:1023500020202020202020207C2020202020202021
:10236000202020202020202020202020202020206D
:10237000202020202020202020202020202020205D
:10238000202020202020202020203220202020203B
:1023900020202020207C7C7C7C20382042697420F6
:1023A00020202020202020207C20202020202020D1
:1023B000202020202020202020202020202020201D
:1023C000202020202020202020202020202020200D
:1023D000202020202020202020207C2020202020A1
:1023E00020202020207C7C7C7C202020202020207D
:1023F00020202020202020207C2020202020202081
:1024000020202020202020202020202020202020CC
:102410002020202020202020202020202020202BB1
:102420002D2D2D2D2D2D2D2B20207C2020202020EA
:1024300020202B2D2D2B2B2B2B2D2B202020202033
:1024400020202020202020207C2020202020202030
:10245000202020202020202020202020202020207C
:102460002020202020202020202020202020207C10
:10247000202020372020207C20207C20202020208D
:1024800020207C202020372020207C20202020207D
:1024900020202020202020207C20202020202020E0
:1024A000202020202020202020202020202020202C
:1024B0002020202020202020202020202020207CC0
:1024C000202020342020207C20207C202020202040
:1024D00020207C202020342020207C202020202030
:1024E00020202020202020207C2020202020202090
:1024F00020202020202020202020202020202020DC
:102500002020202020202020202020202020207C6F
:10251000202020482020207C20207C2020202020DB
:1025200020207C202020482020207C2020202020CB
:1025300020202020202020207C202020202020203F
:10254000202020202020202020202020205647410D
:10255000203C2D2D2D2D2D2D2035202D2D2D2D2BBD
:10256000202020432020202B2D2D2B2D2031202DED
:102570003C2D2B202020432020203C2D2D2D2D2DA7
:102580002D2D2D2D2D2D2D2D2B20202020202020D8
:10259000202020202020202020202020202020203B
:1025A0002020202020202020202020202020207CCF
:1025B000202020322020207C2020202020202020AD
:1025C00020207C202020312020207C202020202042
:1025D00020202020202020202020202020202020FB
:1025E00020202020202020202020202020202020EB
:1025F0002020202020202020202020202020207C7F
:10260000202020342020207C20202020202020205A
:1026100020207C202020362020207C2020202020EC
:1026200020202020202020202020202020202020AA
:10263000202020202020202020202020202020209A
:102640002020202020202020202020202020207C2E
:10265000202020342020207C20202020202020200A
:1026600020207C202020352020207C20202020209D
:10267000202020202020202020202020202020205A
:10268000202020202020202020202020202020204A
:102690002020202020202020202020202020202B2F
:1026A0002D2D2D2D2D2D2D2B2020202020202020C4
:1026B00020202B2D2D2D2D2D2D2D2B2020202020A9
:1026C000202020202020202020202020202020200A
:1026D00020202020202020202020202020202020FA
:1026E00020202020202020202020202020202042C8
:1026F0007573747265696265722020202020202025
:1027000020205363686965626572656769737465E3
:102710007220202020202020202020202020202067
:1027200020202020202020202020202020202020A9
:102730002020202020202020202020202020202099
:102740002020202020202020202020202020202089
:102750002020202020202020202020202020202079
:102760002020202020202020202020202020202069
:102770002020202000202020202020202020202079
:102780002020202020202020202020202020202049
:102790002020202020202020202020202020202039
:1027A0002020202020202020202020202020202029
:1027B0002020202020202020202020202020202019
:1027C00020202020202023232323232320202020F7
:1027D00023232323202020202020202323202023E4
:1027E00023232323202020202020202020202020DD
:1027F00020202020202020202020202020202020D9
:1028000020202020202020202020202020202020C8
:1028100020202020202020232320202323202023A9
:102820002320202323202020202023232020232393
:102830002020202323202020202020202020202092
:102840002020202020202020202020202020202088
:102850002020202020202020202020202020202078
:10286000202020202020202323202023232020205C
:10287000232320202020202020232320202020204C
:102880002020202323202020202020202020202042
:102890002020202020202020202020202020202038
:1028A0002020202020202020202020202020202028
:1028B0002020202020202023232323232020202009
:1028C00020232320202020202323202020202020FC
:1028D00020232323202020202D2054617374617431
:1028E0007572202020202020202020202020202041
:1028F00020202020202020202020202020202020D8
:1029000020202020202020232320202020202020C1
:1029100020202323202020232320202020202020AB
:1029200023232020202020202020202020202020A1
:102930002020202020202020202020202020202097
:102940002020202020202020202020202020202087
:10295000202020202020202323202020202020236E
:102960002320202323202323202020202020202355
:10297000232020232320202020202020202020204E
:102980002020202020202020202020202020202047
:102990002020202020202020202020202020202037
:1029A000202020202020232323232020202020201B
:1029B0002323232320202320202020202020232302
:1029C00023232323232020202020202020202020F8
:1029D00020202020202020202020202020202020F7
:1029E00020202020202020202020202020202020E7
:1029F00020202020202020202020202020202020D7
:102A000020202020202020202020202020202020C6
:102A100020202020202020202020202020202020B6
:102A200020202020202020202020202020202020A6
:102A30002020202020202020202020202020202096
:102A40002020202020202020202020202020202086
:102A50002020202020202020202020202020202076
:102A60002020202020202020202020202020202066
:102A70002020202020202020202020202020202056
:102A80002020202020202020202020202020202046
:102A900020202020202050532F323A2053594E43DB
:102AA00048524F4E45532073657269656C6C65736F
:102AB0002050726F746F6B6F6C6C20202020202070
:102AC0002020202020202020202020202020202006
:102AD00020202020202020202020202020202020F6
:102AE00020202020202020202020202020202020E6
:102AF00020202020202020202020202020202020D6
:102B000020202020202020202020202020202020C5
:102B100020202020202020202020202020202020B5
:102B200020202020202020202020202020202020A5
:102B300020202020202032204C656974756E676546
:102B40006E3A20446174656E20286269646972651A
:102B50006B74696F6E616C2920756E642054616BB3
:102B6000742028696D6D657220766F6E20546173D4
:102B700074617475722065727A6575677429202096
:102B80002020202020202020202020202020202045
:102B90002020202020202020202020202020202035
:102BA0002020202020202020202020202020202025
:102BB0002020202020202020202020202020202015
:102BC0002020202020202020202020202020202005
:102BD00020202020202020202020202020202020F5
:102BE00020202020202020202020202020202020E5
:102BF00020202020202020202020202020202020D5
:102C000020202020202020202020202020202020C4
:102C100020202020202020202020202020202020B4
:102C200020202020202044696520446174656E20A6
:102C300077657264656E20766F6E2054617374617F
:102C4000747572206F646572205043206175662030
:102C5000646572207374656967656E64656E20547F
:102C6000616B74666C616E6B652067657365747A01
:102C70007420202020202020202020202020202000
:102C80002020202020202020202020202020202044
:102C90002020202020202020202020202020202034
:102CA0002020202020202020202020202020202024
:102CB0002020202020202020202020202020202014
:102CC000202020202020756E6420617566206465B8
:102CD000722066616C6C656E64656E20466C616E18
:102CE0006B652067656C6573656E20202020202051
:102CF00020202020202020202020202020202020D4
:102D000020202020202020202020202020202020C3
:102D100020202020202020202020202020202020B3
:102D200020202020202020202020202020202020A3
:102D30002020202020202020202020202020202093
:102D40002020202020202020202020202020202083
:102D50002020202020202020202020202020202073
:102D60002020202020202020202020202020202063
:102D70002020202020202020202020202020202053
:102D80002020202020202020202020202020202043
:102D90002020202020202020202020202020202033
:102DA0002020202020202020202020202020202023
:102DB0002020202020202020202020202020202013
:102DC0002020205F5F5F5F5F5F5F5F5F20202020CC
:102DD00020205F5F5F5F2020202020205F5F5F5FFB
:102DE0002020202020205F5F5F5F202020202020E7
:102DF0005F5F5F5F2020202020205F5F5F5F2020DB
:102E0000202020202020202054616B7420202020AE
:102E10002020202020202020202020207C5F5F5F99
:102E20005F7C202020207C5F5F5F5F7C2020202053
:102E30007C5F5F5F5F7C202020207C5F5F5F5F7C2A
:102E4000202020207C5F5F5F5F7C202020207C5F33
:102E50005F5F5F20202020202020202020202020B5
:102E60002020202020202020202020202020202062
:102E70002020202020202020202020202020202052
:102E80002020202020202020202020202020202042
:102E90002020202020202020202020202020202032
:102EA0002020202020202020202020202020202022
:102EB0002020205F5F5F5F5F5F2020202020202098
:102EC000202020205F5F5F5F5F5F5F5F5F202020CB
:102ED00020202020202020205F5F5F5F5F5F5F5FFA
:102EE0005F5F5F5F5F5F5F5F5F5F5F5F20202020EE
:102EF0002020202020202020446174656E20202086
:102F00002020202020202020207C5F5F5F5F5F5FEB
:102F10005F5F5F7C2020202020202020207C5F5FBE
:102F20005F5F5F5F5F5F5F7C20202020202020208C
:102F30002020202020202020202020207C5F5F5F78
:102F40005F5F5F5F20202020202020202020202085
:102F50002020202020202020202020202020202071
:102F60002020202020202020202020202020202061
:102F70002020202020202020202020202020202051
:102F80002020202020202020202020202020202041
:102F90002020202020202020202020202020202031
:102FA0002020202020202020202020205E202020E3
:102FB0002020202020205E202020202020202020D3
:102FC0005E2020202020202020205E202020202085
:102FD000202020205E2020202020202020205E2075
:102FE00020202020202020202020202020202020E1
:102FF0002020202020202020202020207C20202075
:103000002020202020207C20202020202020202064
:103010007C2020202020202020207C2020202020F8
:10302000202020207C2020202020202020207C20E8
:103030002020202020202020202020202020202090
:103040002020202020202020202020202020202080
:103050002020202020202020202020202020202070
:103060002020202020202020202020202020202060
:103070002020202020202020202020202020202050
:103080002020202020202020202020202020202040
:103090002020202020202020202020203020202020
:1030A000202020202020312020202020202020200F
:1030B00030202020202020202020312020202020EF
:1030C00020202020312020202020202020203020DF
:1030D000202E2E2E202020202020202020202020C6
:1030E00020202020202020202020202020202020E0
:1030F00020202020202020202020202020202020D0
:1031000020202020202020202020202020202020BF
:1031100020202020202020202020202020202020AF
:10312000202020202020202020202020202020209F
:10313000202020202020202020202020202020208F
:10314000202020202020202020202020202020207F
:10315000202020202020202020202020202020206F
:10316000202020202020202020202020202020205F
:10317000202020202020202020312E205461737414
:1031800065202241222067656472FC636B742020F5
:1031900020202020202020203D3E20546173746197
:1031A0007475722073656E646574203078314320C5
:1031B0002020202020736F672E204D616B652D43EA
:1031C0006F64652020202020202020202020202027
:1031D00020202020202020202020202020202020EF
:1031E00020202020202020202020202020202020DF
:1031F00020202020202020202020202020202020CF
:1032000020202020202020202020202020202020BE
:10321000202020202020202020322E205461737472
:103220006520224122206C6F7367656C6173736542
:103230006E202020202020203D3E205461737461A8
:103240007475722073656E64657420307846302022
:103250003143202020736F672E20427265616B2DF1
:10326000436F646520202020202020202020202063
:10327000202020202020202020202020202020204E
:10328000202020202020202020202020202020203E
:10329000202020202020202020202020202020202E
:1032A000202020202020202020202020202020201E
:1032B000202020202020202020332E2054617374D1
:1032C00065202235222067656472FC636B742020C0
:1032D00020202020202020203D3E20546173746156
:1032E0007475722073656E64657420307832452081
:1032F00020202020202020202020202020202020CE
:1033000020202020202020202020202020202020BD
:1033100020202020202020202020202020202020AD
:10332000202020202020202020202020202020209D
:10333000202020202020202020202020202020208D
:10334000202020202020202020202020202020207D
:10335000202020202020202020342E20546173742F
:103360006520223522206C6F7367656C617373650D
:103370006E202020202020203D3E20546173746167
:103380007475722073656E646574203078463020E1
:1033900032452020202020202020202020202020F6
:1033A000202020202020202020202020202020201D
:1033B000202020202020202020202020202020200D
:1033C00020202020202020202020202020202020FD
:1033D00020202020202020202020202020202020ED
:1033E00020202020202020202020202020202020DD
:1033F000202020202020202020352E2052656368A8
:10340000746520506665696C7461737465206765C6
:103410006472FC636B74202020203D3E2054617355
:1034200074617475722073656E64657420307845BC
:103430003020373420202020202020202020202051
:10344000202020202020202020202020202020207C
:10345000202020202020202020202020202020206C
:10346000202020202020202020202020202020205C
:10347000202020202020202020202020202020204C
:10348000202020202020202020202020202020203C
:10349000202020202020202020362E205265636806
:1034A000746520506665696C7461737465206C6F17
:1034B0007367656C617373656E203D3E2054617364
:1034C00074617475722073656E646574203078451C
:1034D000302046302037342020202020202020207B
:1034E00020202020202020202020202020202020DC
:1034F00020202020202020202020202020202020CC
:1035000020202020202020202020202020202020BB
:1035100020202020202020202020202020202020AB
:10352000202020202020202020202020202020209B
:1035300020202020200020202020202020202020AB
:10354000202020202020202020202020202020207B
:10355000202020202020202020202020202020206B
:10356000202020202020202020202020202020205B
:10357000202020202020202020202020202020204B
:10358000202020202020202323202020232320202F
:103590002023232323202020202323232020202016
:1035A000202020202020202020202020202020201B
:1035B00020205653594E433A2076657274696B61E8
:1035C0006C6520202020202020202020202020206A
:1035D00020202020202020232320202023232020DF
:1035E00023232020232320202323202323202020C3
:1035F00020202020202020202020202020202020CB
:103600002020202020202020202842696C642D29A1
:1036100053796E6368726F6E69736174696F6E203F
:10362000202020202020202323202020232320238B
:10363000232020202020202323202020232320207B
:10364000202020202020202020202020202020207A
:10365000202020202020202020202020202020206A
:10366000202020202020202020202020202020205A
:10367000202020202020202323202020232320233B
:103680002320202020202023232323232323202022
:103690002D2042696C646175666261753A20202054
:1036A00020204853594E433A20686F72697A6F6EF2
:1036B00074616C65202020202020202020202020E4
:1036C00020202020202020232320202023232023EB
:1036D00023202023232320232320202023232020D2
:1036E00020202020202020202020202020202020DA
:1036F000202020202020202020285A65696C656E1B
:103700002D2953796E6368726F6E69736174696F86
:103710006E2020202020202023232023232020204F
:103720002323202023232023232020202323202081
:103730002020202020202020202020202020202089
:103740002020202020202020202020202020202079
:103750002020202020202020202020202020202069
:103760002020202020202020202323232020202050
:103770002023232320232023232020202323202031
:103780002020202020202020202020202020202039
:103790002020202020202020202020202020202029
:1037A0002020202020202020202020202020202019
:1037B0002020202020202020202020202020202009
:1037C00020202020202020202020202020202020F9
:1037D00020202020202020202020202020202020E9
:1037E00020202020202020202020202020202020D9
:1037F00020202020202020205653594E43202020D6
:1038000020202020202020202020202020202020B8
:1038100020202020202020202020202020202020A8
:103820002020202020202020202020202020202098
:103830002020202020202020202020202020202088
:103840002020202020202020202020202020202078
:103850002020202020202020202020202020202068
:103860002020202020202020202020202020202058
:103870002020202020202020202020202020202048
:103880002020202020202020202020202020202038
:10389000202020202020202020207C2020202020CC
:1038A0002020202020202020202020202020202018
:1038B0002020202020202020202020202020202008
:1038C00020202020202020202020202020202020F8
:1038D00020202020202020202020202020202020E8
:1038E000202020202020202020207C5F5F202020FE
:1038F00020202020202020202020202020202020C8
:1039000020202020202020202020202020202020B7
:1039100020202020202020202020202020202020A7
:103920002020202020202020202020202020202097
:10393000202020202020202020202020207C20202B
:103940002020202020202020202020202020202077
:1039500020202020202020205F5F5F5F202020206B
:1039600020205F5F5F5F5F5F5F5F5F5F5F5F5F5FE5
:103970005F5F5F5F5F5F5F5F5F5F5F5F5F5F5F5F57
:103980005F5F5F5F5F5F5F5F20202020207C2020E3
:103990002020202020202020202020202020202027
:1039A000204853594E432020202020207C5F5F5F19
:1039B0005F7C20202020202020202020202020206C
:1039C00020202020202020202020202020202020F7
:1039D000202020202020202020202020207C20208B
:1039E000202020202020207363687761727A203C99
:1039F00020202020202020202020202020202020C7
:103A000020202020202020202020202020202020B6
:103A100020202020202020202020202020202020A6
:103A2000202020202020202020202020207C20203A
:103A30002020202020202020202020202020202086
:103A400020522C472C4220205F5F5F5F5F5F5F5FEB
:103A50005F5F5F5F5F5F5F5F5F5F5F5F5F5F5F5F76
:103A60005F5F5F5F5F5F5F5F5F5F5F5F5F5F5F5F66
:103A70005F5F5F5F5F5F5F5F20202020207C2020F2
:103A80002020202020202020202020202020202036
:103A90002020202020202020202020202020202026
:103AA0002020202020202020202020202020202016
:103AB0002020202020202020202020202020202006
:103AC00020202020202020202020205F5F7C2042FA
:103AD000494C44203120202020202020202020205C
:103AE00020202020202020202020202020202020D6
:103AF00020202020202020202020202020202020C6
:103B000020202020202020202020202020202020B5
:103B1000202020202020202020207C202020202049
:103B20002020202020202020202020202020202095
:103B300020202020202020205F5F5F5F2020202089
:103B400020205F5F5F5F5F5F5F5F5F5F5F5F5F5F03
:103B50005F5F5F5F5F5F5F5F5F5F5F5F5F5F5F5F75
:103B60005F5F5F5F5F5F5F5F20207C202020202001
:103B70002020202020202020202020202020202045
:103B8000204853594E432020202020207C5F5F5F37
:103B90005F7C20202020202020202020202020208A
:103BA0002020202020202020202020202020202015
:103BB000202020202020202020207C2020202020A9
:103BC000202020202020205A65696C652031203C6F
:103BD00020202020202020202020202020202020E5
:103BE00020202020202020202020202020202020D5
:103BF00020202020202020202020202020202020C5
:103C0000202020202020202020207C202020202058
:103C100020202020202020202020202020202020A4
:103C200020522C472C4220205F5F5F5F5F5F5F5F09
:103C30005F5F5F5F5F7C7C7C7C7C7C7C7C7C7C7C55
:103C40007C7C7C7C7C7C7C7C7C7C7C7C7C7C7C7CB4
:103C50007C7C7C7C7C7C5F5F20207C202020202062
:103C60002020202020202020202020202020202054
:103C70002020202020202020202020202020202044
:103C80002020202020202020202020202020202034
:103C90002020202020202020202020202020202024
:103CA000202020202020202020207C2020202020B8
:103CB0002020202020202020202020202020202004
:103CC00020202020202020202020202020202020F4
:103CD00020202020202020202020202020202020E4
:103CE00020202020202020202020202020202020D4
:103CF000202020202020202020207C202020202068
:103D000020202020202020202020202020202020B3
:103D100020202020202020205F5F5F5F20202020A7
:103D200020205F5F5F5F5F5F5F5F5F5F5F5F5F5F21
:103D30005F5F5F5F5F5F5F5F5F5F5F5F5F5F5F5F93
:103D40005F5F5F5F5F5F5F5F20207C20202020201F
:103D50002020202020202020202020202020202063
:103D6000204853594E432020202020207C5F5F5F55
:103D70005F7C2020202020202020202020202020A8
:103D80002020202020202020202020202020202033
:103D9000202020202020202020207C2020202020C7
:103DA000202020202020205A65696C652032203C8C
:103DB0002020202020202020202020202020202003
:103DC00020202020202020202020202020202020F3
:103DD00020202020202020202020202020202020E3
:103DE000202020202020202020207C202020202077
:103DF00020202020202020202020202020202020C3
:103E000020522C472C4220205F5F5F5F5F5F5F5F27
:103E10005F5F5F5F5F7C7C7C7C7C7C7C7C7C7C7C73
:103E20007C7C7C7C7C7C7C7C7C7C7C7C7C7C7C7CD2
:103E30007C7C7C7C7C7C5F5F20207C202020202080
:103E40002020202020202020202020202020202072
:103E50002020202020202020202020202020202062
:103E60002020202020202020202020202020202052
:103E70002020202020202020202020202020202042
:103E8000202020202020202020207C2020202020D6
:103E90002020202020202020202020202020202022
:103EA0002020202020202020202020202020202012
:103EB0002020202020202020202020202020202002
:103EC00020202020202020202020202020202020F2
:103ED000202020202020202020207C202020202086
:103EE0002020202020202020202E2E2E20202020A8
:103EF00020202020202020202020202020202020C2
:103F000020202020202020202020202020202020B1
:103F100020202020202020202020202020202020A1
:103F20002020202020202020203D3D3D202020203A
:103F30002020202020202020202020202020202081
:103F40002020202020202020202020202020202071
:103F50002020202020202020202020202020202061
:103F60002020202020202020202020202020202051
:103F7000202020202020202020207C2020202020E5
:103F80002020202020202020202020202020202031
:103F90002020202020202020202020202020202021
:103FA0002020202020202020202020202020202011
:103FB0002020202020202020202020202020202001
:103FC000202020202020202020207C5F5F20202017
:103FD00020202020202020202020202020202020E1
:103FE00020202020202020202020202020202020D1
:103FF00020202020202020202020202020202020C1
:1040000020202020202020202020202020202020B0
:10401000202020202020202020202020207C202044
:104020002020202020202020202020202020202090
:1040300020202020202020205F5F5F5F2020202084
:1040400020205F5F5F5F5F5F5F5F5F5F5F5F5F5FFE
:104050005F5F5F5F5F5F5F5F5F5F5F5F5F5F5F5F70
:104060005F5F5F5F5F5F5F5F20202020207C2020FC
:104070002020202020202020202020202020202040
:10408000204853594E432020202020207C5F5F5F32
:104090005F7C202020202020202020202020202085
:1040A0002020202020202020202020202020202010
:1040B000202020202020202020202020207C2020A4
:1040C000202020202020207363687761727A203CB2
:1040D00020202020202020202020202020202020E0
:1040E00020202020202020202020202020202020D0
:1040F00020202020202020202020202020202020C0
:10410000202020202020202020202020207C202053
:10411000202020202020202020202020202020209F
:1041200020522C472C4220205F5F5F5F5F5F5F5F04
:104130005F5F5F5F5F5F5F5F5F5F5F5F5F5F5F5F8F
:104140005F5F5F5F5F5F5F5F5F5F5F5F5F5F5F5F7F
:104150005F5F5F5F5F5F5F5F20202020207C20200B
:10416000202020202020202020202020202020204F
:10417000202020202020202020202020202020203F
:10418000202020202020202020202020202020202F
:10419000202020202020202020202020202020201F
:1041A00020202020202020202020205F5F7C204213
:1041B000494C442032202020202020202020202074
:1041C00020202020202020202020202020202020EF
:1041D00020202020202020202020202020202020DF
:1041E00020202020202020202020202020202020CF
:1041F000202020202020202020207C202020202063
:1042000020202020202020202020202020202020AE
:1042100020202020202020205F5F5F5F20202020A2
:1042200020205F5F5F5F5F5F5F5F5F5F5F5F5F5F1C
:104230005F5F5F5F5F5F5F5F5F5F5F5F5F5F5F5F8E
:104240005F5F5F5F5F5F5F5F20207C20202020201A
:10425000202020202020202020202020202020205E
:10426000204853594E432020202020207C5F5F5F50
:104270005F7C2020202020202020202020202020A3
:10428000202020202020202020202020202020202E
:10429000202020202020202020207C2020202020C2
:1042A000202020202020205A65696C652031203C88
:1042B00020202020202020202020202020202020FE
:1042C00020202020202020202020202020202020EE
:1042D00020202020202020202020202020202020DE
:1042E000202020202020202020207C202020202072
:1042F00020202020202020202020202020202020BE
:1043000020522C472C4220205F5F5F5F5F5F5F5F22
:104310005F5F5F5F5F7C7C7C7C7C7C7C7C7C7C7C6E
:104320007C7C7C7C7C7C7C7C7C7C7C7C7C7C7C7CCD
:104330007C7C7C7C7C7C5F5F20207C20202020207B
:10434000202020202020202020202020202020206D
:10435000202020202020202020202020202020205D
:10436000202020202020202020202020202020204D
:10437000202020202020202020202020202020203D
:10438000202020202020202020207C2020202020D1
:104390002020202020202020202E2E2E20202020F3
:1043A000202020202020202020202020202020200D
:1043B00020202020202020202020202020202020FD
:1043C00020202020202020202020202020202020ED
:1043D000202020202020202020207C202020202081
:1043E00020202020202000202020202020202020ED
:1043F00020202020202020202020202020202020BD
:1044000020202020202020202020202020202020AC
:10441000202020202020202020202020202020209C
:10442000202020202020202020202020202020208C
:104430002020202020202020232320202023232070
:104440002020232323232020202023232320202057
:10445000202020204461732054696D696E672064B8
:104460006572205647412D5369676E616C6520283F
:104470005653594E432C204853594E432C20522C0E
:1044800020472C20422920202323202020232320C2
:104490002023232020232320202323202323202004
:1044A000202020202020202020202020202020200C
:1044B00020202020202020202020202020202020FC
:1044C00020202020202020202020202020202020EC
:1044D00020202020202020202323202020232320D0
:1044E00023232020202020202323202020232320BA
:1044F0002020202069737420766F6E2064657220FE
:10450000564553412028566964656F20456C6563A4
:1045100074726F6E696373205374616E6461726448
:10452000732020202020202023232020202323202C
:104530002323202020202020232323232323232060
:10454000202020202020202020202020202020206B
:10455000202020202020202020202020202020205B
:10456000202020202020202020202020202020204B
:10457000202020202020202023232020202323202F
:104580002323202023232320232320202023232010
:10459000202020204173736F63696174696F6E29F5
:1045A000206665737467656C6567742E2020202013
:1045B00020202020202020202020202020202020FB
:1045C00020202020202020202023232023232020DF
:1045D00020232320202323202323202020232320C3
:1045E00020202020202020202020202020202020CB
:1045F00020202020202020202020202020202020BB
:1046000020202020202020202020202020202020AA
:104610002020202020202020202023232320202091
:104620002020232323202320232320202023232072
:10463000202020202020202020202020202020207A
:10464000202020202020202020202020202020206A
:10465000202020202020202020202020202020205A
:10466000202020202020202020202020202020204A
:10467000202020202020202020202020202020203A
:10468000202020202020202020202020202020202A
:10469000202020202020202020202020202020201A
:1046A000202020202020202020202020202020200A
:1046B00020202020202020202020202020202020FA
:1046C00020202020202020202020202020202020EA
:1046D00020202020202020202020202020202020DA
:1046E00020202020202020202020202020202020CA
:1046F00020202020202020202020202020202020BA
:1047000020202020202020202020202020202020A9
:104710002020202020202020202020202020202099
:104720002020202020202020202020202020202089
:104730002020202020202020202020202020202079
:104740002020202020202020202020202020202069
:1047500020202020202020202020417566626175C5
:104760002065696E657220566964656F2D5A4549EA
:104770004C453A20202020202020202020202020CE
:104780002020202020202020202020202020202029
:104790002020202020202020202020202020202019
:1047A0002020202020202020202020202020202009
:1047B00020202020202020202020202020202020F9
:1047C00020202020202020202020202020202020E9
:1047D00020202020202020202020202020202020D9
:1047E00020202020202020202020202020202020C9
:1047F00020202020202020202020202020202020B9
:1048000020202020205F5F5F5F2020202020205F6D
:104810005F5F5F5F5F5F5F5F5F5F5F5F5F5F5F5FA8
:104820005F5F5F5F5F5F5F5F5F5F5F5F5F5F5F5F98
:104830005F5F5F5F5F5F5F5F5F5F5F5F5F5F5F5F88
:104840005F5F5F5F5F5F202020204853594E432009
:104850002020202020202020207C5F5F5F5F7C20A4
:104860002020202020202020202020202020202048
:104870002020202020202020202020202020202038
:104880002020202020202020202020202020202028
:104890002020202020202020202020202020202018
:1048A0002020202020202020202020202020202008
:1048B00020202020202020202020202020202020F8
:1048C00020202020202020202020202020202020E8
:1048D00020202020202020202020202020202020D8
:1048E00020202020202020202020202020202020C8
:1048F00020202020202020202020202020202020B8
:1049000020202020205F2020205F2020205F2020EA
:10491000205F2020205F2020205F2020205F20209B
:10492000205F2020205F2020205F2020205F20208B
:10493000205F2020202020202020522C472C4220A5
:1049400020202020205F5F5F5F5F5F5F5F5F5F5FB2
:104950005F5F5F5F7C207C5F7C207C5F7C207C5F76
:104960007C207C5F7C207C5F7C207C5F7C207C5F6B
:104970007C207C5F7C207C5F7C207C5F7C207C5F5B
:104980007C207C5F5F5F20202020202020202020B2
:104990002020202020202020202020202020202017
:1049A0002020202020202020202020202020202007
:1049B00020202020202020202020202020202020F7
:1049C00020202020202020202020202020202020E7
:1049D00020202020202020202020202020202020D7
:1049E00020202020202020202020202020202020C7
:1049F00020202020202020202020202020202020B7
:104A000020202020202020202020202020202020A6
:104A10002020202020202020202020202020202096
:104A20002020202020202020202020202020202086
:104A300020202020203C2D2D3E2020202020202022
:104A4000202020202020202020202020766F72642B
:104A5000657265205363687761727A736368756CF9
:104A6000746572202866726F6E7420706F7263684E
:104A7000292020202020202020202020202020202D
:104A80002020202020202020202020202020202026
:104A90002020202020202020202020202020202016
:104AA0002020202020202020202020202020202006
:104AB00020202020202020202020202020202020F6
:104AC00020202020202020202020202020202020E6
:104AD0002020202020202020203C2D2D2D2D3E2068
:104AE00020202020202020202020202053796E63A9
:104AF00068726F6E69736174696F6E732D50756C37
:104B0000732028686F722E2073796E63292020200D
:104B10002020202020202020202020202020202095
:104B20002020202020202020202020202020202085
:104B30002020202020202020202020202020202075
:104B40002020202020202020202020202020202065
:104B50002020202020202020202020202020202055
:104B60002020202020202020202020202020202045
:104B70002020202020202020202020202020203C19
:104B80002D2D2D3E202020202020202068696E74AD
:104B9000657265205363687761727A736368756CB8
:104BA00074657220286261636B20706F726368297C
:104BB00020202020202020202020202020202020F5
:104BC00020202020202020202020202020202020E5
:104BD00020202020202020202020202020202020D5
:104BE00020202020202020202020202020202020C5
:104BF00020202020202020202020202020202020B5
:104C000020202020202020202020202020202020A4
:104C10002020202020202020202020202020202094
:104C2000202020203C2D2D2D2D202020736963680D
:104C300074626172657220426572656963682028DA
:104C400061637469766520766964656F2920202D1B
:104C50002D2D2D2D2D3E20202020202020202020F5
:104C60002020202020202020202020202020202044
:104C70002020202020202020202020202020202034
:104C80002020202020202020202020202020202024
:104C90002020202020202020202020202020202014
:104CA0002020202020202020202020202020202004
:104CB00020202020202020202020202020202020F4
:104CC00020202020202020202020202020202020E4
:104CD00020202020202020202020202020202020D4
:104CE00020202020202020202020202020202020C4
:104CF00020202020202020202020202020202020B4
:104D000020202020202020202020202020202020A3
:104D10002020202020202020202020202020202093
:104D20002020202020202020202020202020202083
:104D30002020202020202020202020202020202073
:104D40002020202020202020202020202020202063
:104D50002020202020202020202020202020202053
:104D60002020202020202020202020202020202043
:104D70002020202020202020202020202020202033
:104D80002020202020202020202020202020202023
:104D9000202020202020202020204175666261757F
:104DA0002065696E657320566964656F2D42494CB4
:104DB000447320286672616D65293A2020202020E6
:104DC00020202020202020202020202020202020E3
:104DD00020202020202020202020202020202020D3
:104DE00020202020202020202020202020202020C3
:104DF00020202020202020202020202020202020B3
:104E000020202020202020202020202020202020A2
:104E10002020202020202020202020202020202092
:104E20002020202020202020202020202020202082
:104E30002020202020202020202020202020202072
:104E40002020202020202020202020205F5F5F5F66
:104E50005F5F5F5F5F5F5F5F5F202020202020201B
:104E60002020202020202020202020202020202042
:104E70002020202020202020202020202020202032
:104E8000202020202020202020205653594E43202F
:104E90002020202020205F5F5F5F5F7C202020207B
:104EA0002020202020202020207C5F5F5F5F5F5F2C
:104EB0005F5F5F5F5F5F5F5F5F5F5F5F5F5F5F5F02
:104EC0005F5F5F5F5F5F5F5F5F5F5F5F5F5F5F5FF2
:104ED0005F5F5F5F5F5F2020202020202020202058
:104EE00020202020202020202020202020202020C2
:104EF00020202020202020202020202020202020B2
:104F000020202020202020202020202020202020A1
:104F10002020202020202020202020202020202091
:104F20002020202020202020202020202020202081
:104F30002020202020205F2020205F5F5F5F202036
:104F4000205F5F5F5F2020205F5F5F5F2020205F2A
:104F50005F5F5F2020205F5F5F5F2020205F5F5FDB
:104F60005F2020205F5F5F5F2020205F5F5F5F200A
:104F700020205F5F5F5F202020204853594E432050
:104F8000202020202020207C5F7C202020207C5F8F
:104F90007C202020207C5F7C202020207C5F7C20C7
:104FA0002020207C5F7C202020207C5F7C20202013
:104FB000207C5F7C202020207C5F7C202020207CA7
:104FC0005F7C202020202020202020202020202046
:104FD00020202020202020202020202020202020D1
:104FE00020202020202020202020202020202020C1
:104FF00020202020202020202020202020202020B1
:1050000020202020202020202020202020202020A0
:105010002020202020202020202020202020202090
:1050200020202020202020202020205F5F20202002
:1050300020205F5F20202020205F5F202020202074
:105040005F5F20202020205F5F20202020205F5FE6
:1050500020202020205F5F20202020205F5F202054
:105060002020205F5F2020202020522C472C42202F
:1050700020202020205F5F5F5F5F7C20207C5F5FBF
:105080005F7C20207C5F5F5F7C20207C5F5F5F7C9B
:1050900020207C5F5F5F7C20207C5F5F5F7C202026
:1050A0007C5F5F5F7C20207C5F5F5F7C20207C5F7B
:1050B0005F5F7C20207C20202020202020202020BA
:1050C00020202020202020202020202020202020E0
:1050D00020202020202020202020202020202020D0
:1050E00020202020202020202020202020202020C0
:1050F00020202020202020202020202020202020B0
:105100002020202020202000741875273635E74302
:1051100011241FBECFEFD0E1DEBFCDBF11E0A0E074
:10512000B1E0EEE6FEE502C005900D92A630B107B3
:10513000D9F710E1A6E0B1E001C01D92A43EB1078D
:10514000E1F70E94E82A0C94352F0C9400001F927E
:105150000F920FB60F9211248F938091110181301D
:1051600069F0813018F0823021F510C05F9A8BE42D
:105170008093B30081E08093120105C05F9885E9B8
:105180008093B30082E08093100115C01092120149
:105190008091B1008B7F8093B10084E28093B30053
:1051A0001092B20084E086BB80916F00846080938F
:1051B0006F001092100180911001809311018F9166
:1051C0000F900FBE0F901F9018951F920F920FB661
:1051D0000F9211242F934F935F936F937F938F932D
:1051E0009F93CF93DF93EF93FF9340910E015091E4
:1051F0000F0181E040395807A9F482E291E09093D1
:1052000004018093030110920F0110920E0180910E
:105210006F008B7F80936F008091B10084608093DA
:10522000B1003CC0242F27706091030170910401EC
:10523000E0E0F0E888E090E0EB01F20F0C944A2BFC
:10524000273031F4605B7F4F70930401609303015A
:105250004F5F5F4F50930F0140930E018091C0004C
:1052600087FF0CC08091D310E82FF0E09091C6002A
:10527000EC52FF4E90838F5F8093D3108091C800D3
:1052800087FF0CC08091C210E82FF0E09091CE0013
:10529000ED53FF4E90838F5F8093C210FF91EF918B
:1052A000DF91CF919F918F917F916F915F914F91FE
:1052B0002F910F900FBE0F901F90189580910B01AA
:1052C0008F5F80930B01843009F07EC010920B0138
:1052D00020910C012F5F20930C0121508AEF95E063
:1052E0004FEC5CE0FC01EE5DFE4F2083FA01E81B11
:1052F000F90BEE5DFE4F208301962F5F36E086337B
:10530000930781F790910101E92FF0E0EE50F74FFC
:1053100080E2808320910201920F90930101E92F96
:10532000F0E0EE50F74F82E08083963418F021953C
:10533000209302019A3028F4809102018195809394
:1053400002018091090190910A01019690930A014E
:10535000809309018A5B914020F010920A0110921B
:1053600009018091090190910A019C0153E0220FEB
:10537000331F5A95E1F7880F991F280F391F205DB9
:10538000384F65E47AE01BC09F5FFA01EE5DFE4F87
:105390008081FA01EF5DFE4F80834F5F5F4F953450
:1053A00099F7F9018491FB01EE5DFE4F80832F5F39
:1053B0003F4F605B7F4FFDE065367F0729F0AB0113
:1053C0004A5350409AE0E0CF08950E94D32D80EADE
:1053D00095E020E3FC01EE5DFE4F2083FC01EF58D9
:1053E000FE4F2083805B9F4F2F5F203599F78FEF13
:1053F0006CE14DEB50E00E94DF2D8AE16DE240EA66
:1054000050E00E94DF2D8FEF60E34CE750E00E94F8
:10541000DF2D82E291E06FE272E00E94252F089575
:10542000DF93CF9300D0CDB7DEB7909108012091E4
:10543000070130E036C0E32FF0E0ED53FF4EE0818E
:10544000E03E69F1222371F0E43729F49F5F943044
:1054500038F193E025C0EB3629F49150943000F1F7
:1054600090E01EC0EC3251F49093080110920701B5
:1054700081E0809306010E94D32D0CC0EB3411F023
:1054800020E00EC0909308011092070110920601CF
:105490000E94E52980E060E00E94242D37C021E0D1
:1054A0003F5F8091C210381730F29093080120932B
:1054B00007011092C210809100019817C9F00E9454
:1054C000D32D6091080170E0660F771F685F7E4AF8
:1054D000CE01019642E050E00E941C2F69817A8142
:1054E00082E291E00E94252F8091080180930001C3
:1054F0008AE061E34BEF50E00E94DF2D80910801CC
:105500008F5C8093821084E3809386100F900F90BD
:10551000CF91DF91089580910D018F5F80930D01F0
:105520008C3021F410920D010E944F2D08951F938D
:105530000E948B2A10E008C0E12FF0E0EC52FF4EF1
:1055400080810E94362E1F5F8091D3101817A0F320
:105550001092D31010E008C0E12FF0E0ED53FF4EA1
:1055600080810E94702E1F5F8091C2101817A0F3D7
:105570001092C2101F91089580910601813011F19F
:10558000813018F0823019F520C08091C210882334
:10559000A1F0E091C210F0E0EE53FF4E808189321D
:1055A00061F482E0809306010E94D32D80E060E0E8
:1055B0000E94242D1092C21008951092C2100E94D1
:1055C0005E2908950E94972A08950E94102A08953E
:1055D0000E94E5298FEF81B912B884B1886184B93E
:1055E00088E085B9559A579A1092810028E1209356
:1055F000810082EC8093800084E080936F0083E6DA
:1056000090E0909387008093860087E090E09093ED
:1056100089008093880088E090E090938B008093CD
:105620008A0010928500109284001092B10082E0EE
:105630008093B000809370001092B20083E080935A
:10564000B3001092C0002093C10086E08093C20096
:1056500082EA90E09093C5008093C4000E94532E8C
:1056600078948091810082608093810083B7817FEC
:1056700083BF83B7816083BF7894889583B78E7F1B
:1056800083BF809112018823A1F30E94BC2A10924B
:105690001201EFCFE991049002B815B885B9E991EC
:1056A000049002B815B885B9E991049002B815B80C
:1056B00085B9E991049002B815B885B9E9910490CB
:1056C00002B815B885B9E991049002B815B885B942
:1056D000E991049002B815B885B9E991049002B82F
:1056E00015B885B9E991049002B815B885B9E99162
:1056F000049002B815B885B9E991049002B815B8BC
:1057000085B9E991049002B815B885B9E99104907A
:1057100002B815B885B9E991049002B815B885B9F1
:10572000E991049002B815B885B9E991049002B8DE
:1057300015B885B9E991049002B815B885B9E99111
:10574000049002B815B885B9E991049002B815B86B
:1057500085B9E991049002B815B885B9E99104902A
:1057600002B815B885B9E991049002B815B885B9A1
:10577000E991049002B815B885B9E991049002B88E
:1057800015B885B9E991049002B815B885B9E991C1
:10579000049002B815B885B9E991049002B815B81B
:1057A00085B9E991049002B815B885B9E9910490DA
:1057B00002B815B885B9E991049002B815B885B951
:1057C000E991049002B815B885B9E991049002B83E
:1057D00015B885B9E991049002B815B885B9E99171
:1057E000049002B815B885B9E991049002B815B8CB
:1057F00085B9E991049002B815B885B9E99104908A
:1058000002B815B885B9E991049002B815B885B900
:10581000E991049002B815B885B9E991049002B8ED
:1058200015B885B9E991049002B815B885B9E99120
:10583000049002B815B885B9E991049002B815B87A
:1058400085B9E991049002B815B885B9E991049039
:1058500002B815B885B9E991049002B815B885B9B0
:10586000E991049002B815B885B9E991049002B89D
:1058700015B885B9E991049002B815B885B9E991D0
:10588000049002B815B885B9E991049002B815B82A
:1058900085B9E991049002B815B885B9E9910490E9
:1058A00002B815B885B9E991049002B815B885B960
:1058B000E991049002B815B885B9E991049002B84D
:1058C00015B885B9E991049002B815B885B9E99180
:1058D000049002B815B885B9E991049002B815B8DA
:1058E00085B9E991049002B815B885B9E991049099
:1058F00002B815B885B9E991049002B815B885B910
:10590000E991049002B815B885B9E991049002B8FC
:1059100015B885B9E991049002B815B885B9E9912F
:10592000049002B815B885B9E991049002B815B889
:1059300085B9E991049002B815B885B9E991049048
:1059400002B815B885B9E991049002B815B885B9BF
:10595000E991049002B815B885B9E991049002B8AC
:1059600015B885B9E991049002B815B885B9E991DF
:10597000049002B815B885B9E991049002B815B839
:1059800085B9E991049002B815B885B9E9910490F8
:1059900002B815B885B9E991049002B815B885B96F
:1059A000E991049002B815B885B9E991049002B85C
:1059B00015B885B90C942029809117018F5F8093C9
:1059C000170180911701803539F4809118018F5F9C
:1059D000809318011092170180911801823369F4A5
:1059E00080E090E0FC01EE5DFE4F108201962FE01A
:1059F000803A9207B9F7109218010895E0911801C2
:105A00009091170180E5E89FF0011124E90FF11D45
:105A1000EE5DFE4F1082809118018F5F8093180118
:105A20001092170180911801823369F480E090E0B0
:105A3000FC01EE5DFE4F108201962FE0803A920746
:105A4000B9F7109218010895809317016093180117
:105A500008959091190190931B01909117019093D3
:105A600019018093170180911A0180931C01809184
:105A7000180180931A01609318010895809119010B
:105A80008093170180911B018093190180911A0165
:105A90008093180180911C0180931A0108958091D0
:105AA00015018823D1F02091140180911701281746
:105AB00089F49091130180911801981759F48091FD
:105AC0001601E0E59E9FF0011124E20FF11DEE5D4D
:105AD000FE4F8083109215010895E0911801809186
:105AE000170190E5E99FF0011124E80FF11DEE5D2B
:105AF000FE4F808180931601E0911801809117017B
:105B0000E99FF0011124E80FF11DEE5DFE4F82E0E8
:105B100080838091170180931401809118018093F4
:105B2000130181E0809315010895E09118012091FF
:105B3000170190E5E99FF0011124E20FF11DEE5DE0
:105B4000FE4F80830895E09118019091170180E540
:105B5000E89FF0011124E90FF11DEE5DFE4F8081F9
:105B600008950F931F93CF93DF93EC0110E000E5AE
:105B70000EC0E091180180911701E09FF0011124FF
:105B8000E80FF11DEE5DFE4F90830E94DC2CFE01BC
:105B9000E10FF11D1F5F9491992359F7DF91CF9188
:105BA0001F910F91089580E090E0FC01EE5DFE4FA3
:105BB000108201962FE0803A9207B9F708950F936B
:105BC0001F93CF93DF93282F162FEA01809119019D
:105BD00080931B0180911701809319011092170186
:105BE00080911A0180931C018091180180931A0101
:105BF000109218012F3F49F4CA010E942C2F20E572
:105C000030E0281B390B3695279520931701109308
:105C1000180110E000E50EC0E09118018091170115
:105C2000E09FF0011124E80FF11DEE5DFE4F90831F
:105C30000E94DC2CFE01E10FF11D1F5F949199235E
:105C400059F7809119018093170180911B0180936E
:105C5000190180911A018093180180911C01809391
:105C60001A01DF91CF911F910F91089590911D011D
:105C7000992319F0913081F408958B3121F481E05A
:105C800080931D0108958A3019F40E94FE2C089516
:105C90008D3021F40000089510921D010E94952D71
:105CA0000E94DC2C08951092C80080E18093C90006
:105CB00086E48093CA001092C21010921F010895CA
:105CC0001F93182F8A3019F40E94FE2C04C00E94E2
:105CD000952D0E94DC2C812F0E94142F1F91089576
:105CE0001F93182F80911E01882399F0103E11F008
:105CF00010921E0110922001123129F0193519F06D
:105D0000113131F503C010921F0122C01092210100
:105D10001FC0183591F0193528F41131B1F0123146
:105D2000C9F40BC0103E69F0103F19F0193591F419
:105D300004C081E080931E010BC081E080931F01AD
:105D400007C081E08093200103C081E0809321019E
:105D500080E068C080912001882349F080E00E94A3
:105D6000602E812F0E94602E109220015AC08091D7
:105D700021018823D1F030E001C03F5F432F50E084
:105D8000440F551FCA01895E9D4FFC0124912117C4
:105D900011F0222391F7FC018491811709F041C091
:105DA000485E5D4FFA0184913AC080911F018823BB
:105DB00011F030E01AC030E001C03F5F432F50E0E7
:105DC000440F551FCA01895F9E4FFC012491211782
:105DD00011F0222391F7FC0184918117E1F4485FCF
:105DE0005E4FFA0184911BC03F5F432F50E0440F88
:105DF000551FCA0181579E4FFC012491211711F0B4
:105E0000222391F7FC018491811729F440575E4FBA
:105E1000FA01849104C080E00E94602E812F0E94CC
:105E2000602E81E01F910895982F8091C00085FF1A
:105E3000FCCF9093C6000895FB01DC0102C00590E1
:105E40000D9241505040D8F70895FB01DC010590B8
:105E50000D920020E1F70895FC0105900020E9F77C
:0E5E6000809590958E0F9F1F0895F894FFCFA8
:065E6E00FF0A0122010001
:10800000007E7E6C10381000FF00FF0F3C3F7F9910
:10801000800218667F7E001818180000000000001B
:1080200000306C6C30003860186000000000000602
:10803000783078781CFC38FC78780000180060787C
:108040007C30FC3CFCFEFE3CCC781EE6F0C6C6381C
:10805000FC78FC78FCCCCCC6C6CCFE78C07810008E
:108060003000E0001C003800E03018E07000000034
:1080700000000000100000000000001C18E0761056
:1080800078001C7ECCE030007ECCE0CC7CE0CC30B4
:108090001C003E780000780000C6CC1838CCF00EEA
:1080A0001C38000000FC3C3C300000C6C60000004C
:1080B0002255DD18181836000036360036361800FE
:1080C0001818001800181836360036003600361812
:1080D0003600003618000036181800FF00F00FFFB9
:1080E00000000000FE000000FC38381C00063C7850
:1080F000003060180E1830003800000F787800004B
:108100000081FFFE387C1000FF3CC3076633635AD2
:10811000E00E3C66DBC3003C3C181830002418FF1E
:1081200000786C6C7CC66C60303066300000000CEF
:10813000CCF0CCCC3CC060CCCCCC0000300030CCFF
:10814000C67866666C626266CC300C6660EEE66C81
:1081500066CC66CCB4CCCCC6C6CCCC60601838003B
:10816000300060000C006C00600000603000000017
:108170000000000030000000000000301830DC3843
:10818000CCCC00C300003000C3000000C60030307B
:1081900000006CCCCCE0CCE0CC3800186CCCD81B08
:1081A00000001C1CF8006C66000000CCCC1833CC1E
:1081B00088AA7718181836000036360036361800A8
:1081C0001818001800181836360036003600361811
:1081D0003600003618000036181800FF00F00FFFB8
:1081E0000078FEFE66006676306C6C30000C60CC69
:1081F000FC3030301B1830726C00000C6C0C00002E
:1082000000A5DBFE7C383818E766990F663F7F3C97
:10821000F83E7E66DB78007E7E180C60C0663CFF10
:1082200000786CFEC0CC38C060183C3000000018EC
:10823000DC300C0C6CF8C00CCCCC303060FC180C72
:10824000DECC66C0666868C0CC300C6C60FEF6C6DA
:1082500066CC66E030CCCCC66CCC986030186C0034
:1082600018787C780C7860766C70786630ECF878EA
:10827000DC76D87C7CCCCCC6C6CCFC301830006C0C
:10828000C000783C7878787C3C78787038707800DA
:10829000FC7FCC0000000000007CCC7E6478D81805
:1082A0007870000000CC6C66300000D8D80066669C
:1082B0002255DD1818F83600F8F636FEF636F800C6
:1082C0001818001800181F36373FF7FF37FFF7FF61
:1082D00036FF00361F1F0036FF1800FF00F00FFFAB
:1082E00076CCC66C307E66DC78C6C6187E7EC0CC86
:1082F00000FC18601B18009C6C00000C6C383C00E3
:108300000081FFFEFEFE7C3CC342BD7D663063E71C
:10831000FEFE18667BCC00181818FEFEC0FF7E7E9D
:108320000030006C781876006018FFFC00FC00300C
:10833000FC303838CC0CF818787C3030C0000C1881
:10834000DECC7CC0667878C0FC300C7860D6DEC6A7
:108350007CCC7C3830CCCCD6387830601818C6004D
:10836000000C66CC7CCCF0CC7630186C30FECCCCDB
:1083700066CC6CC030CCCCC66CCC98E0001C00C67F
:10838000CCCCCC060C0C0CC066CCCC301830CC78E5
:10839000600CFE787878CCCCCCC6CCC0F0FCF47EF7
:1083A0000C3078CCF8EC3E3C60FCFC3EF318CC334F
:1083B00088AA7718181836001806360606361800E8
:1083C000181800180018183630300000300000006F
:1083D0003600003618180036001800FF00F00FFFB6
:1083E000DCF8C06C18CC6618CCFEC67CDBDBFCCCA1
:1083F000FC3030301818FC003818000C6C603C0061
:1084000000BDC37C7CFEFE3CC342BDCC3C3063E778
:10841000F83E18661BCC7E7E187E0C60C066FF3C62
:10842000003000FE0C30DC0060183C3000000060C2
:10843000EC30600CFE0CCC30CC0C000060FC183032
:10844000DEFC66C0666868CECC30CC6C62C6CEC638
:1084500060DC781C30CCCCFE6C3062600C18000004
:10846000007C66C0CCFC60CC6630187830D6CCCCB2
:1084700066CC6C7830CCCCD638CC3030183000C6D6
:1084800078CCFC3E7C7C7CC07EFCFC301830CCCCB4
:10849000787FCCCCCCCCCCCCCCC6CCC06030CC188B
:1084A0007C30CCCCCCFC0000C0C00C636718666686
:1084B0002255DD18F8F8F6FEF8F636F6FEFEF8F866
:1084C0001FFFFF1FFFFF1F373F37FFF737FFF7FF84
:1084D000FFFFFF3F1F1F3FF7FFF81FFFFFF00F00D9
:1084E000C8CCC06C30CC6618CCC66CCCDBDBC0CC46
:1084F0000030601818180072001818EC6C7C3C00F2
:108500000099E73838D67C18E76699CC1870673C34
:10851000E00E7E001B787E3C183C1830FE24FF18CD
:108520000000006CF866CC0030306630700030C05F
:10853000CC30CCCC0CCCCC60CC18307030003000BF
:10854000C0CC66666C626066CC30CC6666C6C66CB3
:1085500060786CCC30CC78EEC630C660061800006F
:1085600000CC66CCCCC0607C6630186C30C6CCCCFD
:108570007C7C600C34CC78FE6C7C6430183000C697
:1085800018CCC066CCCCCC7C60C0C0301830FCFCB1
:1085900060CCCCCCCCCCCCCCFC7CCC7EE6FCDE184D
:1085A000CC30CCCCCCDC7E7ECCC00CCECF3C33CC23
:1085B00088AA77181818363618363636000000188C
:1085C000000018180018183600360036360036003D
:1085D0000018360000183636180018FFFFF00F009C
:1085E000DCF8C06C66CC7C18786C6CCC7E7E60CC81
:1085F000FC00000018D8309C0000006C00003C001B
:108600000081FF1010101000FF3CC3CC7EF0E65A32
:1086100080023C661B8C7E181818000000000000C9
:108620000030006C30C676001860000030003080EA
:1086300078FCFC780C787860787030301800603006
:1086400078CCFC3CFCFEF03ECC7878E6FEC6C63822
:10865000F01CE67878FC30C6C678FE780278000018
:108660000076BC787678F00CE678D8E678C6CC78D8
:10867000600CF0F81876306CC60CFC1C18E000FE9C
:108680000C7E783F7E7E7E063C7878783C78CCCC39
:10869000FC7FCE7878787E7E0C387818FC30CCD889
:1086A0007E78787ECCCC0000780000989F3C00005B
:1086B0002255DD18181836361836363600000018E0
:1086C000000018180018183600360036360036003C
:1086D0000018360000183636180018FFFFF00F009B
:1086E00076C0C06CFE7860183038EE7800603CCC04
:1086F00000FCFCFC18D830000000003C000000002A
:10870000007E7E0000383800FF00FF7818E0C09936
:108710000000180000F800FF00000000000000004A
:1087200000000000000000000000000060000000E9
:1087300000000000000000000000006000000000D9
:108740000000000000000000000000000000000029
:10875000000000000000000000000000000000FF1A
:1087600000000000000000F80000700000000000A1
:10877000F01E00000000000000F8000000000000F3
:10878000780000000000003C000000000000000035
:108790000000000000000000F800001800000E704B
:1087A00000000000000000000000001F031800008F
:1087B00088AA77181818363618363636000000188A
:1087C000000018180018183600360036360036003B
:1087D0000018360000183636180018FFFFF00F009A
:1087E00000C000000000C000FC00000000C000004D
:1087F00000000000187000000000001C00000000D5
:00000001FF
